:0100000000FF
:0100010000FE
:0100020000FD
:0100030000FC
:0100040000FB
:0100050000FA
:0100060000F9
:0100070000F8
:0100080000F7
:0100090000F6
:01000A0000F5
:01000B0000F4
:01000C0000F3
:01000D0000F2
:01000E0000F1
:01000F0000F0
:0100100000EF
:0100110000EE
:0100120000ED
:0100130000EC
:0100140000EB
:0100150000EA
:0100160000E9
:0100170000E8
:0100180000E7
:0100190000E6
:01001A0000E5
:01001B0000E4
:01001C0000E3
:01001D0000E2
:01001E0000E1
:01001F0000E0
:0100200000DF
:0100210000DE
:0100220000DD
:0100230000DC
:0100240000DB
:0100250000DA
:0100260000D9
:0100270000D8
:0100280000D7
:0100290000D6
:01002A0000D5
:01002B0000D4
:01002C0000D3
:01002D0000D2
:01002E0000D1
:01002F0000D0
:0100300000CF
:0100310000CE
:0100320000CD
:0100330000CC
:0100340000CB
:0100350000CA
:0100360000C9
:0100370000C8
:0100380000C7
:0100390000C6
:01003A0000C5
:01003B0000C4
:01003C0000C3
:01003D0000C2
:01003E0000C1
:01003F0000C0
:0100400000BF
:0100410000BE
:0100420000BD
:0100430000BC
:0100440000BB
:0100450000BA
:0100460000B9
:0100470000B8
:0100480000B7
:0100490000B6
:01004A0000B5
:01004B0000B4
:01004C0000B3
:01004D0000B2
:01004E0000B1
:01004F0000B0
:0100500000AF
:0100510000AE
:0100520000AD
:0100530000AC
:0100540000AB
:0100550000AA
:0100560000A9
:0100570000A8
:0100580000A7
:0100590000A6
:01005A0000A5
:01005B0000A4
:01005C0000A3
:01005D0000A2
:01005E0000A1
:01005F0000A0
:01006000009F
:01006100009E
:01006200009D
:01006300009C
:01006400009B
:01006500009A
:010066000099
:010067000098
:010068000097
:010069000096
:01006A000095
:01006B000094
:01006C000093
:01006D000092
:01006E000091
:01006F000090
:01007000008F
:01007100008E
:01007200008D
:01007300008C
:01007400008B
:01007500008A
:010076000089
:010077000088
:010078000087
:010079000086
:01007A000085
:01007B000084
:01007C000083
:01007D000082
:01007E000081
:01007F000080
:01008000007F
:01008100007E
:01008200007D
:01008300007C
:01008400007B
:01008500007A
:010086000079
:010087000078
:010088000077
:010089000076
:01008A000075
:01008B000074
:01008C000073
:01008D000072
:01008E000071
:01008F000070
:01009000006F
:01009100006E
:01009200006D
:01009300006C
:01009400006B
:01009500006A
:010096000069
:010097000068
:010098000067
:010099000066
:01009A000065
:01009B000064
:01009C000063
:01009D000062
:01009E000061
:01009F000060
:0100A000005F
:0100A100005E
:0100A200005D
:0100A300005C
:0100A400005B
:0100A500005A
:0100A6000059
:0100A7000058
:0100A8000057
:0100A9000056
:0100AA000055
:0100AB000054
:0100AC000053
:0100AD000052
:0100AE000051
:0100AF000050
:0100B000004F
:0100B100004E
:0100B200004D
:0100B300004C
:0100B400004B
:0100B500004A
:0100B6000049
:0100B7000048
:0100B8000047
:0100B9000046
:0100BA000045
:0100BB000044
:0100BC000043
:0100BD000042
:0100BE000041
:0100BF000040
:0100C000003F
:0100C100003E
:0100C200003D
:0100C300003C
:0100C400003B
:0100C500003A
:0100C6000039
:0100C7000038
:0100C8000037
:0100C9000036
:0100CA000035
:0100CB000034
:0100CC000033
:0100CD000032
:0100CE000031
:0100CF000030
:0100D000002F
:0100D100002E
:0100D200002D
:0100D300002C
:0100D400002B
:0100D500002A
:0100D6000029
:0100D7000028
:0100D8000027
:0100D9000026
:0100DA000025
:0100DB000024
:0100DC000023
:0100DD000022
:0100DE000021
:0100DF000020
:0100E000001F
:0100E100001E
:0100E200001D
:0100E300001C
:0100E400001B
:0100E500001A
:0100E6000019
:0100E7000018
:0100E8000017
:0100E9000016
:0100EA000015
:0100EB000014
:0100EC000013
:0100ED000012
:0100EE000011
:0100EF000010
:0100F000000F
:0100F100000E
:0100F200000D
:0100F300000C
:0100F400000B
:0100F500000A
:0100F6000009
:0100F7000008
:0100F8000007
:0100F9000006
:0100FA000005
:0100FB000004
:0100FC000003
:0100FD000002
:0100FE000001
:0100FF000000
:0101000000FE
:0101010000FD
:0101020000FC
:0101030000FB
:0101040000FA
:0101050000F9
:0101060000F8
:0101070000F7
:0101080000F6
:0101090000F5
:01010A0000F4
:01010B0000F3
:01010C0000F2
:01010D0000F1
:01010E0000F0
:01010F0000EF
:0101100000EE
:0101110000ED
:0101120000EC
:0101130000EB
:0101140000EA
:0101150000E9
:0101160000E8
:0101170000E7
:0101180000E6
:0101190000E5
:01011A0000E4
:01011B0000E3
:01011C0000E2
:01011D0000E1
:01011E0000E0
:01011F0000DF
:0101200000DE
:0101210000DD
:0101220000DC
:0101230000DB
:0101240000DA
:0101250000D9
:0101260000D8
:0101270000D7
:0101280000D6
:0101290000D5
:01012A0000D4
:01012B0000D3
:01012C0000D2
:01012D0000D1
:01012E0000D0
:01012F0000CF
:0101300000CE
:0101310000CD
:0101320000CC
:0101330000CB
:0101340000CA
:0101350000C9
:0101360000C8
:0101370000C7
:0101380000C6
:0101390000C5
:01013A0000C4
:01013B0000C3
:01013C0000C2
:01013D0000C1
:01013E0000C0
:01013F0000BF
:0101400000BE
:0101410000BD
:0101420000BC
:0101430000BB
:0101440000BA
:0101450000B9
:0101460000B8
:0101470000B7
:0101480000B6
:0101490000B5
:01014A0000B4
:01014B0000B3
:01014C0000B2
:01014D0000B1
:01014E0000B0
:01014F0000AF
:0101500000AE
:0101510000AD
:0101520000AC
:0101530000AB
:0101540000AA
:0101550000A9
:0101560000A8
:0101570000A7
:0101580000A6
:0101590000A5
:01015A0000A4
:01015B0000A3
:01015C0000A2
:01015D0000A1
:01015E0000A0
:01015F00009F
:01016000009E
:01016100009D
:01016200009C
:01016300009B
:010164000199
:010165000198
:010166000197
:010167000196
:010168000195
:010169000194
:01016A000193
:01016B000192
:01016C000191
:01016D000190
:01016E00018F
:01016F00018E
:01017000018D
:01017100018C
:01017200018B
:01017300018A
:010174000189
:010175000188
:010176000187
:010177000186
:010178000185
:010179000184
:01017A000183
:01017B000182
:01017C000181
:01017D000180
:01017E00017F
:01017F00017E
:01018000017D
:01018100017C
:01018200017B
:01018300017A
:010184000179
:010185000178
:010186000177
:010187000176
:010188000175
:010189000174
:01018A000173
:01018B000172
:01018C000171
:01018D000170
:01018E00016F
:01018F00016E
:01019000016D
:01019100016C
:01019200016B
:01019300016A
:010194000169
:010195000168
:010196000167
:010197000166
:010198000165
:010199000164
:01019A000163
:01019B000162
:01019C000161
:01019D000160
:01019E00015F
:01019F00015E
:0101A000015D
:0101A100005D
:0101A200005C
:0101A300005B
:0101A400005A
:0101A5000059
:0101A6000058
:0101A7000057
:0101A8000056
:0101A9000055
:0101AA000153
:0101AB00054E
:0101AC00054D
:0101AD00054C
:0101AE00054B
:0101AF00054A
:0101B0000549
:0101B100014C
:0101B200014B
:0101B300014A
:0101B4000149
:0101B5000148
:0101B6000147
:0101B7000146
:0101B8000145
:0101B9000144
:0101BA000143
:0101BB000142
:0101BC000141
:0101BD000140
:0101BE00013F
:0101BF00013E
:0101C000013D
:0101C100013C
:0101C200013B
:0101C300013A
:0101C4000139
:0101C5000138
:0101C6000137
:0101C7000136
:0101C8000135
:0101C9000134
:0101CA000133
:0101CB000132
:0101CC000131
:0101CD000130
:0101CE00012F
:0101CF00012E
:0101D000012D
:0101D100012C
:0101D200012B
:0101D300012A
:0101D4000129
:0101D5000128
:0101D6000127
:0101D7000126
:0101D8000125
:0101D9000124
:0101DA000123
:0101DB000122
:0101DC000121
:0101DD000120
:0101DE00011F
:0101DF00051A
:0101E000011D
:0101E100011C
:0101E200011B
:0101E300011A
:0101E4000515
:0101E5000514
:0101E6000117
:0101E7000017
:0101E8000016
:0101E9000015
:0101EA000014
:0101EB000013
:0101EC000012
:0101ED000011
:0101EE000010
:0101EF00000F
:0101F000010D
:0101F1000508
:0101F200010B
:0101F300010A
:0101F4000109
:0101F5000108
:0101F6000503
:0101F7000106
:0101F8000105
:0101F9000104
:0101FA000103
:0101FB000102
:0101FC000101
:0101FD000100
:0101FE0001FF
:0101FF0001FE
:0102000001FC
:0102010001FB
:0102020001FA
:0102030001F9
:0102040001F8
:0102050001F7
:0102060001F6
:0102070001F5
:0102080001F4
:0102090001F3
:01020A0001F2
:01020B0001F1
:01020C0001F0
:01020D0001EF
:01020E0001EE
:01020F0001ED
:0102100001EC
:0102110001EB
:0102120001EA
:0102130001E9
:0102140001E8
:0102150001E7
:0102160001E6
:0102170001E5
:0102180001E4
:0102190001E3
:01021A0001E2
:01021B0001E1
:01021C0001E0
:01021D0001DF
:01021E0001DE
:01021F0001DD
:0102200001DC
:0102210001DB
:0102220001DA
:0102230001D9
:0102240001D8
:0102250005D3
:0102260005D2
:0102270005D1
:0102280005D0
:0102290005CF
:01022A0005CE
:01022B0005CD
:01022C0001D0
:01022D0000D0
:01022E0000CF
:01022F0000CE
:0102300000CD
:0102310000CC
:0102320000CB
:0102330000CA
:0102340000C9
:0102350000C8
:0102360001C6
:0102370005C1
:0102380005C0
:0102390005BF
:01023A0005BE
:01023B0005BD
:01023C0005BC
:01023D0001BF
:01023E0001BE
:01023F0001BD
:0102400001BC
:0102410001BB
:0102420001BA
:0102430001B9
:0102440001B8
:0102450001B7
:0102460001B6
:0102470001B5
:0102480001B4
:0102490001B3
:01024A0001B2
:01024B0001B1
:01024C0001B0
:01024D0001AF
:01024E0001AE
:01024F0001AD
:0102500001AC
:0102510001AB
:0102520001AA
:0102530001A9
:0102540001A8
:0102550001A7
:0102560001A6
:0102570001A5
:0102580001A4
:0102590001A3
:01025A0001A2
:01025B0001A1
:01025C0001A0
:01025D00019F
:01025E00019E
:01025F00019D
:01026000019C
:01026100019B
:01026200019A
:010263000199
:010264000198
:010265000197
:010266000196
:010267000195
:010268000194
:010269000193
:01026A000192
:01026B00058D
:01026C000190
:01026D00018F
:01026E00018E
:01026F00018D
:01027000018C
:01027100018B
:01027200018A
:01027300008A
:010274000089
:010275000088
:010276000087
:010277000086
:010278000085
:010279000084
:01027A000083
:01027B000082
:01027C000180
:01027D00017F
:01027E00017E
:01027F00017D
:01028000017C
:01028100017B
:010282000675
:010283000674
:010284000673
:010285000672
:010286000671
:010287000670
:01028800066F
:01028900066E
:01028A00066D
:01028B00066C
:01028C00066B
:01028D00066A
:01028E000669
:01028F000668
:010290000667
:010291000666
:010292000665
:010293000664
:010294000663
:010295000662
:010296000661
:010297000660
:01029800065F
:01029900065E
:01029A00065D
:01029B00065C
:01029C00065B
:01029D00065A
:01029E000659
:01029F000658
:0102A0000657
:0102A1000656
:0102A2000655
:0102A3000654
:0102A4000653
:0102A5000652
:0102A6000651
:0102A7000650
:0102A800064F
:0102A900064E
:0102AA00064D
:0102AB00064C
:0102AC00064B
:0102AD00064A
:0102AE000649
:0102AF000648
:0102B0000647
:0102B1000646
:0102B2000645
:0102B3000149
:0102B4000148
:0102B5000147
:0102B6000146
:0102B7000145
:0102B8000144
:0102B9000044
:0102BA000043
:0102BB000042
:0102BC000041
:0102BD000040
:0102BE00003F
:0102BF00003E
:0102C000003D
:0102C100003C
:0102C200013A
:0102C3000139
:0102C4000138
:0102C5000137
:0102C6000136
:0102C7000135
:0102C800062F
:0102C9000331
:0102CA000330
:0102CB00032F
:0102CC00032E
:0102CD00032D
:0102CE00032C
:0102CF00032B
:0102D000032A
:0102D1000329
:0102D2000328
:0102D3000327
:0102D4000326
:0102D5000325
:0102D6000324
:0102D7000323
:0102D8000322
:0102D9000321
:0102DA000320
:0102DB00031F
:0102DC00031E
:0102DD00031D
:0102DE00031C
:0102DF00041A
:0102E0000419
:0102E1000418
:0102E2000417
:0102E3000416
:0102E4000415
:0102E5000414
:0102E6000413
:0102E7000412
:0102E8000411
:0102E9000410
:0102EA00040F
:0102EB00040E
:0102EC00040D
:0102ED00040C
:0102EE00040B
:0102EF00040A
:0102F0000409
:0102F1000408
:0102F2000407
:0102F3000406
:0102F4000405
:0102F5000404
:0102F6000403
:0102F7000402
:0102F80006FF
:0102F9000103
:0102FA000102
:0102FB000101
:0102FC000100
:0102FD0001FF
:0102FE0001FE
:0102FF0000FE
:0103000000FC
:0103010000FB
:0103020000FA
:0103030000F9
:0103040000F8
:0103050000F7
:0103060000F6
:0103070000F5
:0103080001F3
:0103090001F2
:01030A0001F1
:01030B0001F0
:01030C0001EF
:01030D0001EE
:01030E0006E8
:01030F0003EA
:0103100003E9
:0103110003E8
:0103120003E7
:0103130003E6
:0103140003E5
:0103150003E4
:0103160003E3
:0103170003E2
:0103180003E1
:0103190003E0
:01031A0003DF
:01031B0003DE
:01031C0003DD
:01031D0003DC
:01031E0003DB
:01031F0003DA
:0103200003D9
:0103210003D8
:0103220003D7
:0103230003D6
:0103240003D5
:0103250004D3
:0103260004D2
:0103270004D1
:0103280004D0
:0103290004CF
:01032A0004CE
:01032B0004CD
:01032C0004CC
:01032D0004CB
:01032E0004CA
:01032F0004C9
:0103300004C8
:0103310004C7
:0103320004C6
:0103330004C5
:0103340004C4
:0103350004C3
:0103360004C2
:0103370004C1
:0103380004C0
:0103390004BF
:01033A0004BE
:01033B0004BD
:01033C0004BC
:01033D0004BB
:01033E0006B8
:01033F0001BC
:0103400001BB
:0103410001BA
:0103420001B9
:0103430001B8
:0103440001B7
:0103450000B7
:0103460000B6
:0103470000B5
:0103480000B4
:0103490000B3
:01034A0000B2
:01034B0000B1
:01034C0000B0
:01034D0000AF
:01034E0001AD
:01034F0001AC
:0103500001AB
:0103510001AA
:0103520001A9
:0103530001A8
:0103540006A2
:0103550003A4
:0103560003A3
:0103570003A2
:0103580003A1
:0103590003A0
:01035A00039F
:01035B00039E
:01035C00039D
:01035D00039C
:01035E00039B
:01035F00039A
:010360000399
:010361000398
:010362000397
:010363000396
:010364000395
:010365000394
:010366000393
:010367000392
:010368000391
:010369000390
:01036A00038F
:01036B00048D
:01036C00048C
:01036D00048B
:01036E00048A
:01036F000489
:010370000488
:010371000487
:010372000486
:010373000485
:010374000484
:010375000483
:010376000482
:010377000481
:010378000480
:01037900047F
:01037A00047E
:01037B00047D
:01037C00047C
:01037D00047B
:01037E00047A
:01037F000479
:010380000478
:010381000477
:010382000476
:010383000475
:010384000672
:010385000176
:010386000175
:010387000174
:010388000173
:010389000172
:01038A000171
:01038B000071
:01038C000070
:01038D00006F
:01038E00006E
:01038F00006D
:01039000006C
:01039100006B
:01039200006A
:010393000069
:010394000167
:010395000166
:010396000165
:010397000164
:010398000163
:010399000162
:01039A00065C
:01039B00035E
:01039C00035D
:01039D00035C
:01039E00035B
:01039F00035A
:0103A0000359
:0103A1000358
:0103A2000357
:0103A3000752
:0103A4000751
:0103A5000750
:0103A600074F
:0103A700074E
:0103A8000351
:0103A9000350
:0103AA00034F
:0103AB00034E
:0103AC00034D
:0103AD00034C
:0103AE00034B
:0103AF00034A
:0103B0000349
:0103B1000447
:0103B2000446
:0103B3000445
:0103B4000444
:0103B5000443
:0103B6000442
:0103B7000441
:0103B8000440
:0103B900043F
:0103BA00043E
:0103BB000839
:0103BC000838
:0103BD000837
:0103BE000836
:0103BF000835
:0103C0000438
:0103C1000437
:0103C2000436
:0103C3000435
:0103C4000434
:0103C5000433
:0103C6000432
:0103C7000431
:0103C8000430
:0103C900042F
:0103CA00062C
:0103CB000130
:0103CC00012F
:0103CD00012E
:0103CE00012D
:0103CF00012C
:0103D000012B
:0103D100002B
:0103D200002A
:0103D3000029
:0103D4000028
:0103D5000027
:0103D6000026
:0103D7000025
:0103D8000024
:0103D9000023
:0103DA000121
:0103DB000120
:0103DC00011F
:0103DD00011E
:0103DE00011D
:0103DF00011C
:0103E0000616
:0103E1000318
:0103E2000317
:0103E3000316
:0103E4000315
:0103E5000314
:0103E6000313
:0103E7000312
:0103E8000311
:0103E900070C
:0103EA00070B
:0103EB00070A
:0103EC000709
:0103ED000708
:0103EE00030B
:0103EF00030A
:0103F0000309
:0103F1000308
:0103F2000307
:0103F3000306
:0103F4000305
:0103F5000304
:0103F6000303
:0103F7000401
:0103F8000400
:0103F90004FF
:0103FA0004FE
:0103FB0004FD
:0103FC0004FC
:0103FD0004FB
:0103FE0004FA
:0103FF0004F9
:0104000004F7
:0104010008F2
:0104020008F1
:0104030008F0
:0104040008EF
:0104050008EE
:0104060004F1
:0104070004F0
:0104080004EF
:0104090004EE
:01040A0004ED
:01040B0004EC
:01040C0004EB
:01040D0004EA
:01040E0004E9
:01040F0004E8
:0104100006E5
:0104110001E9
:0104120001E8
:0104130001E7
:0104140001E6
:0104150001E5
:0104160001E4
:0104170000E4
:0104180000E3
:0104190000E2
:01041A0000E1
:01041B0000E0
:01041C0000DF
:01041D0000DE
:01041E0000DD
:01041F0000DC
:0104200001DA
:0104210001D9
:0104220001D8
:0104230001D7
:0104240001D6
:0104250001D5
:0104260006CF
:0104270003D1
:0104280003D0
:0104290003CF
:01042A0003CE
:01042B0003CD
:01042C0003CC
:01042D0003CB
:01042E0003CA
:01042F0007C5
:0104300007C4
:0104310007C3
:0104320007C2
:0104330007C1
:0104340003C4
:0104350003C3
:0104360003C2
:0104370003C1
:0104380003C0
:0104390003BF
:01043A0003BE
:01043B0003BD
:01043C0003BC
:01043D0004BA
:01043E0004B9
:01043F0004B8
:0104400004B7
:0104410004B6
:0104420004B5
:0104430004B4
:0104440004B3
:0104450004B2
:0104460004B1
:0104470008AC
:0104480008AB
:0104490008AA
:01044A0008A9
:01044B0008A8
:01044C0004AB
:01044D0004AA
:01044E0004A9
:01044F0004A8
:0104500004A7
:0104510004A6
:0104520004A5
:0104530004A4
:0104540004A3
:0104550004A2
:01045600069F
:0104570001A3
:0104580001A2
:0104590001A1
:01045A0001A0
:01045B00019F
:01045C00019E
:01045D00009E
:01045E00009D
:01045F00009C
:01046000009B
:01046100009A
:010462000099
:010463000098
:010464000097
:010465000096
:010466000194
:010467000193
:010468000192
:010469000191
:01046A000190
:01046B00018F
:01046C000689
:01046D00038B
:01046E00038A
:01046F000389
:010470000388
:010471000387
:010472000386
:010473000385
:010474000384
:01047500077F
:01047600077E
:01047700077D
:01047800077C
:01047900077B
:01047A00037E
:01047B00037D
:01047C00037C
:01047D00037B
:01047E00037A
:01047F000379
:010480000378
:010481000377
:010482000376
:010483000474
:010484000473
:010485000472
:010486000471
:010487000470
:01048800046F
:01048900046E
:01048A00046D
:01048B00046C
:01048C00046B
:01048D000866
:01048E000865
:01048F000864
:010490000863
:010491000862
:010492000465
:010493000464
:010494000463
:010495000462
:010496000461
:010497000460
:01049800045F
:01049900045E
:01049A00045D
:01049B00045C
:01049C000659
:01049D00015D
:01049E00015C
:01049F00015B
:0104A000015A
:0104A1000159
:0104A2000158
:0104A3000058
:0104A4000057
:0104A5000056
:0104A6000055
:0104A7000054
:0104A8000053
:0104A9000052
:0104AA000051
:0104AB000050
:0104AC00014E
:0104AD00014D
:0104AE00014C
:0104AF00014B
:0104B000014A
:0104B1000149
:0104B2000643
:0104B3000345
:0104B4000344
:0104B5000343
:0104B6000342
:0104B7000341
:0104B8000340
:0104B900033F
:0104BA00033E
:0104BB000739
:0104BC000738
:0104BD000737
:0104BE000736
:0104BF000735
:0104C0000338
:0104C1000337
:0104C2000336
:0104C3000335
:0104C4000334
:0104C5000333
:0104C6000332
:0104C7000331
:0104C8000330
:0104C900042E
:0104CA00042D
:0104CB00042C
:0104CC00042B
:0104CD00042A
:0104CE000429
:0104CF000428
:0104D0000427
:0104D1000426
:0104D2000425
:0104D3000820
:0104D400081F
:0104D500081E
:0104D600081D
:0104D700081C
:0104D800041F
:0104D900041E
:0104DA00041D
:0104DB00041C
:0104DC00041B
:0104DD00041A
:0104DE000419
:0104DF000418
:0104E0000417
:0104E1000416
:0104E2000613
:0104E3000117
:0104E4000116
:0104E5000115
:0104E6000114
:0104E7000113
:0104E8000112
:0104E9000012
:0104EA000011
:0104EB000010
:0104EC00000F
:0104ED00000E
:0104EE00000D
:0104EF00000C
:0104F000000B
:0104F100000A
:0104F2000108
:0104F3000107
:0104F4000106
:0104F5000105
:0104F6000104
:0104F7000103
:0104F80006FD
:0104F90003FF
:0104FA0003FE
:0104FB0003FD
:0104FC0003FC
:0104FD0003FB
:0104FE0003FA
:0104FF0003F9
:0105000003F7
:0105010007F2
:0105020007F1
:0105030007F0
:0105040007EF
:0105050007EE
:0105060003F1
:0105070003F0
:0105080003EF
:0105090003EE
:01050A0003ED
:01050B0003EC
:01050C0003EB
:01050D0003EA
:01050E0003E9
:01050F0004E7
:0105100004E6
:0105110004E5
:0105120004E4
:0105130004E3
:0105140004E2
:0105150004E1
:0105160004E0
:0105170004DF
:0105180004DE
:0105190008D9
:01051A0008D8
:01051B0008D7
:01051C0008D6
:01051D0008D5
:01051E0004D8
:01051F0004D7
:0105200004D6
:0105210004D5
:0105220004D4
:0105230004D3
:0105240004D2
:0105250004D1
:0105260004D0
:0105270004CF
:0105280006CC
:0105290001D0
:01052A0001CF
:01052B0001CE
:01052C0001CD
:01052D0001CC
:01052E0001CB
:01052F0000CB
:0105300000CA
:0105310000C9
:0105320000C8
:0105330000C7
:0105340000C6
:0105350000C5
:0105360000C4
:0105370000C3
:0105380001C1
:0105390001C0
:01053A0001BF
:01053B0001BE
:01053C0001BD
:01053D0001BC
:01053E0006B6
:01053F0003B8
:0105400003B7
:0105410003B6
:0105420003B5
:0105430003B4
:0105440003B3
:0105450003B2
:0105460003B1
:0105470003B0
:0105480003AF
:0105490003AE
:01054A0003AD
:01054B0003AC
:01054C0003AB
:01054D0003AA
:01054E0003A9
:01054F0003A8
:0105500003A7
:0105510003A6
:0105520003A5
:0105530003A4
:0105540003A3
:0105550004A1
:0105560004A0
:01055700049F
:01055800049E
:01055900049D
:01055A00049C
:01055B00049B
:01055C00049A
:01055D000499
:01055E000498
:01055F000497
:010560000496
:010561000495
:010562000494
:010563000493
:010564000492
:010565000491
:010566000490
:01056700048F
:01056800048E
:01056900048D
:01056A00048C
:01056B00048B
:01056C00048A
:01056D000489
:01056E000686
:01056F00018A
:010570000189
:010571000188
:010572000187
:010573000186
:010574000185
:010575000085
:010576000084
:010577000083
:010578000082
:010579000081
:01057A000080
:01057B00007F
:01057C00007E
:01057D00007D
:01057E00017B
:01057F00017A
:010580000179
:010581000178
:010582000177
:010583000176
:010584000670
:010585000372
:010586000371
:010587000370
:01058800036F
:01058900036E
:01058A00036D
:01058B00036C
:01058C00036B
:01058D00036A
:01058E000369
:01058F000368
:010590000367
:010591000366
:010592000365
:010593000364
:010594000363
:010595000362
:010596000361
:010597000360
:01059800035F
:01059900035E
:01059A00035D
:01059B00045B
:01059C00045A
:01059D000459
:01059E000458
:01059F000457
:0105A0000456
:0105A1000455
:0105A2000454
:0105A3000453
:0105A4000452
:0105A5000451
:0105A6000450
:0105A700044F
:0105A800044E
:0105A900044D
:0105AA00044C
:0105AB00044B
:0105AC00044A
:0105AD000449
:0105AE000448
:0105AF000447
:0105B0000446
:0105B1000445
:0105B2000444
:0105B3000443
:0105B4000640
:0105B5000144
:0105B6000143
:0105B7000142
:0105B8000141
:0105B9000140
:0105BA00013F
:0105BB00003F
:0105BC00003E
:0105BD00003D
:0105BE00003C
:0105BF00003B
:0105C000003A
:0105C1000039
:0105C2000038
:0105C3000037
:0105C4000135
:0105C5000134
:0105C6000133
:0105C7000132
:0105C8000131
:0105C9000130
:0105CA00062A
:0105CB00032C
:0105CC00032B
:0105CD00032A
:0105CE000329
:0105CF000328
:0105D0000327
:0105D1000326
:0105D2000325
:0105D3000324
:0105D4000323
:0105D5000322
:0105D6000321
:0105D7000320
:0105D800031F
:0105D900031E
:0105DA00031D
:0105DB00031C
:0105DC00031B
:0105DD00031A
:0105DE000319
:0105DF000318
:0105E0000317
:0105E1000415
:0105E2000414
:0105E3000413
:0105E4000412
:0105E5000411
:0105E6000410
:0105E700040F
:0105E800040E
:0105E900040D
:0105EA00040C
:0105EB00040B
:0105EC00040A
:0105ED000409
:0105EE000408
:0105EF000407
:0105F0000406
:0105F1000405
:0105F2000404
:0105F3000403
:0105F4000402
:0105F5000401
:0105F6000400
:0105F70004FF
:0105F80004FE
:0105F90004FD
:0105FA0006FA
:0105FB0001FE
:0105FC0001FD
:0105FD0001FC
:0105FE0001FB
:0105FF0001FA
:0106000001F8
:0106010000F8
:0106020000F7
:0106030000F6
:0106040000F5
:0106050000F4
:0106060000F3
:0106070000F2
:0106080000F1
:0106090000F0
:01060A0001EE
:01060B0001ED
:01060C0001EC
:01060D0001EB
:01060E0001EA
:01060F0001E9
:0106100006E3
:0106110006E2
:0106120006E1
:0106130006E0
:0106140006DF
:0106150006DE
:0106160006DD
:0106170006DC
:0106180006DB
:0106190006DA
:01061A0006D9
:01061B0006D8
:01061C0006D7
:01061D0006D6
:01061E0006D5
:01061F0006D4
:0106200006D3
:0106210006D2
:0106220006D1
:0106230006D0
:0106240006CF
:0106250006CE
:0106260006CD
:0106270006CC
:0106280006CB
:0106290006CA
:01062A0006C9
:01062B0006C8
:01062C0006C7
:01062D0006C6
:01062E0006C5
:01062F0006C4
:0106300006C3
:0106310006C2
:0106320006C1
:0106330006C0
:0106340006BF
:0106350006BE
:0106360006BD
:0106370006BC
:0106380006BB
:0106390006BA
:01063A0006B9
:01063B0006B8
:01063C0006B7
:01063D0006B6
:01063E0006B5
:01063F0006B4
:0106400006B3
:0106410001B7
:0106420001B6
:0106430001B5
:0106440001B4
:0106450001B3
:0106460001B2
:0106470000B2
:0106480000B1
:0106490000B0
:01064A0000AF
:01064B0000AE
:01064C0000AD
:01064D0000AC
:01064E0000AB
:01064F0000AA
:0106500001A8
:0106510005A3
:0106520005A2
:0106530005A1
:0106540005A0
:01065500059F
:01065600059E
:0106570001A1
:0106580001A0
:01065900019F
:01065A00019E
:01065B00019D
:01065C00019C
:01065D00019B
:01065E00019A
:01065F000199
:010660000198
:010661000197
:010662000196
:010663000195
:010664000194
:010665000193
:010666000192
:010667000191
:010668000190
:01066900018F
:01066A00018E
:01066B00018D
:01066C00018C
:01066D00018B
:01066E00018A
:01066F000189
:010670000188
:010671000187
:010672000186
:010673000185
:010674000184
:010675000183
:010676000182
:010677000181
:010678000180
:01067900017F
:01067A00017E
:01067B00017D
:01067C00017C
:01067D00017B
:01067E00017A
:01067F000179
:010680000178
:010681000177
:010682000176
:010683000175
:010684000174
:01068500056F
:010686000172
:010687000171
:010688000170
:01068900016F
:01068A00056A
:01068B000569
:01068C00016C
:01068D00006C
:01068E00006B
:01068F00006A
:010690000069
:010691000068
:010692000067
:010693000066
:010694000065
:010695000064
:010696000162
:01069700055D
:010698000160
:01069900015F
:01069A00015E
:01069B00015D
:01069C000558
:01069D00015B
:01069E00015A
:01069F000159
:0106A0000158
:0106A1000157
:0106A2000156
:0106A3000155
:0106A4000154
:0106A5000153
:0106A6000152
:0106A7000151
:0106A8000150
:0106A900014F
:0106AA00014E
:0106AB00014D
:0106AC00014C
:0106AD00014B
:0106AE00014A
:0106AF000149
:0106B0000148
:0106B1000147
:0106B2000146
:0106B3000145
:0106B4000144
:0106B5000143
:0106B6000142
:0106B7000141
:0106B8000140
:0106B900013F
:0106BA00013E
:0106BB00013D
:0106BC00013C
:0106BD00013B
:0106BE00013A
:0106BF000139
:0106C0000138
:0106C1000137
:0106C2000136
:0106C3000135
:0106C4000134
:0106C5000133
:0106C6000132
:0106C7000131
:0106C8000130
:0106C900012F
:0106CA00012E
:0106CB000529
:0106CC000528
:0106CD000527
:0106CE000526
:0106CF000525
:0106D0000524
:0106D1000523
:0106D2000126
:0106D3000026
:0106D4000025
:0106D5000024
:0106D6000023
:0106D7000022
:0106D8000021
:0106D9000020
:0106DA00001F
:0106DB00001E
:0106DC00011C
:0106DD000517
:0106DE000516
:0106DF000515
:0106E0000514
:0106E1000513
:0106E2000512
:0106E3000115
:0106E4000114
:0106E5000113
:0106E6000112
:0106E7000111
:0106E8000110
:0106E900010F
:0106EA00010E
:0106EB00010D
:0106EC00010C
:0106ED00010B
:0106EE00010A
:0106EF000109
:0106F0000108
:0106F1000107
:0106F2000106
:0106F3000105
:0106F4000104
:0106F5000103
:0106F6000102
:0106F7000101
:0106F8000100
:0106F90001FF
:0106FA0001FE
:0106FB0001FD
:0106FC0001FC
:0106FD0001FB
:0106FE0001FA
:0106FF0001F9
:0107000001F7
:0107010001F6
:0107020001F5
:0107030001F4
:0107040001F3
:0107050001F2
:0107060001F1
:0107070001F0
:0107080001EF
:0107090001EE
:01070A0001ED
:01070B0001EC
:01070C0001EB
:01070D0001EA
:01070E0001E9
:01070F0001E8
:0107100001E7
:0107110005E2
:0107120001E5
:0107130001E4
:0107140001E3
:0107150001E2
:0107160001E1
:0107170001E0
:0107180001DF
:0107190000DF
:01071A0000DE
:01071B0000DD
:01071C0000DC
:01071D0000DB
:01071E0000DA
:01071F0000D9
:0107200000D8
:0107210000D7
:0107220001D5
:0107230001D4
:0107240001D3
:0107250001D2
:0107260001D1
:0107270001D0
:0107280001CF
:0107290001CE
:01072A0001CD
:01072B0001CC
:01072C0001CB
:01072D0001CA
:01072E0001C9
:01072F0001C8
:0107300001C7
:0107310001C6
:0107320001C5
:0107330001C4
:0107340001C3
:0107350001C2
:0107360001C1
:0107370001C0
:0107380001BF
:0107390001BE
:01073A0001BD
:01073B0001BC
:01073C0001BB
:01073D0001BA
:01073E0001B9
:01073F0001B8
:0107400001B7
:0107410001B6
:0107420001B5
:0107430001B4
:0107440001B3
:0107450001B2
:0107460001B1
:0107470001B0
:0107480001AF
:0107490001AE
:01074A0001AD
:01074B0001AC
:01074C0001AB
:01074D0001AA
:01074E0001A9
:01074F0001A8
:0107500001A7
:0107510001A6
:0107520001A5
:0107530001A4
:0107540001A3
:0107550001A2
:0107560001A1
:0107570001A0
:01075800019F
:01075900019E
:01075A00019D
:01075B00019C
:01075C00019B
:01075D00019A
:01075E000199
:01075F000099
:010760000098
:010761000097
:010762000096
:010763000095
:010764000094
:010765000093
:010766000092
:010767000091
:010768000090
:01076900008F
:01076A00008E
:01076B00008D
:01076C00008C
:01076D00008B
:01076E00008A
:01076F000089
:010770000088
:010771000087
:010772000086
:010773000085
:010774000084
:010775000083
:010776000082
:010777000081
:010778000080
:01077900007F
:01077A00007E
:01077B00007D
:01077C00007C
:01077D00007B
:01077E00007A
:01077F000079
:010780000078
:010781000077
:010782000076
:010783000075
:010784000074
:010785000073
:010786000072
:010787000071
:010788000070
:01078900006F
:01078A00006E
:01078B00006D
:01078C00006C
:01078D00006B
:01078E00006A
:01078F000069
:010790000068
:010791000067
:010792000066
:010793000065
:010794000064
:010795000063
:010796000062
:010797000061
:010798000060
:01079900005F
:01079A00005E
:01079B00005D
:01079C00005C
:01079D00005B
:01079E00005A
:01079F000059
:0107A0000058
:0107A1000057
:0107A2000056
:0107A3000055
:0107A4000054
:0107A5000053
:0107A6000052
:0107A7000051
:0107A8000050
:0107A900004F
:0107AA00004E
:0107AB00004D
:0107AC00004C
:0107AD00004B
:0107AE00004A
:0107AF000049
:0107B0000048
:0107B1000047
:0107B2000046
:0107B3000045
:0107B4000044
:0107B5000043
:0107B6000042
:0107B7000041
:0107B8000040
:0107B900003F
:0107BA00003E
:0107BB00003D
:0107BC00003C
:0107BD00003B
:0107BE00003A
:0107BF000039
:0107C0000038
:0107C1000037
:0107C2000036
:0107C3000035
:0107C4000034
:0107C5000033
:0107C6000032
:0107C7000031
:0107C8000030
:0107C900002F
:0107CA00002E
:0107CB00002D
:0107CC00002C
:0107CD00002B
:0107CE00002A
:0107CF000029
:0107D0000028
:0107D1000027
:0107D2000026
:0107D3000025
:0107D4000024
:0107D5000023
:0107D6000022
:0107D7000021
:0107D8000020
:0107D900001F
:0107DA00001E
:0107DB00001D
:0107DC00001C
:0107DD00001B
:0107DE00001A
:0107DF000019
:0107E0000018
:0107E1000017
:0107E2000016
:0107E3000015
:0107E4000014
:0107E5000013
:0107E6000012
:0107E7000011
:0107E8000010
:0107E900000F
:0107EA00000E
:0107EB00000D
:0107EC00000C
:0107ED00000B
:0107EE00000A
:0107EF000009
:0107F0000008
:0107F1000007
:0107F2000006
:0107F3000005
:0107F4000004
:0107F5000003
:0107F6000002
:0107F7000001
:0107F8000000
:0107F90000FF
:0107FA0000FE
:0107FB0000FD
:0107FC0000FC
:0107FD0000FB
:0107FE0000FA
:0107FF0000F9
:0108000000F7
:0108010000F6
:0108020000F5
:0108030000F4
:0108040000F3
:0108050000F2
:0108060000F1
:0108070000F0
:0108080000EF
:0108090000EE
:01080A0000ED
:01080B0000EC
:01080C0000EB
:01080D0000EA
:01080E0000E9
:01080F0000E8
:0108100000E7
:0108110000E6
:0108120000E5
:0108130000E4
:0108140000E3
:0108150000E2
:0108160000E1
:0108170000E0
:0108180000DF
:0108190000DE
:01081A0000DD
:01081B0000DC
:01081C0000DB
:01081D0000DA
:01081E0000D9
:01081F0000D8
:0108200000D7
:0108210000D6
:0108220000D5
:0108230000D4
:0108240000D3
:0108250000D2
:0108260000D1
:0108270000D0
:0108280000CF
:0108290000CE
:01082A0000CD
:01082B0000CC
:01082C0000CB
:01082D0000CA
:01082E0000C9
:01082F0000C8
:0108300000C7
:0108310000C6
:0108320000C5
:0108330000C4
:0108340000C3
:0108350000C2
:0108360000C1
:0108370000C0
:0108380000BF
:0108390000BE
:01083A0000BD
:01083B0000BC
:01083C0000BB
:01083D0000BA
:01083E0000B9
:01083F0000B8
:0108400000B7
:0108410000B6
:0108420000B5
:0108430000B4
:0108440000B3
:0108450000B2
:0108460000B1
:0108470000B0
:0108480000AF
:0108490000AE
:01084A0000AD
:01084B0000AC
:01084C0000AB
:01084D0000AA
:01084E0000A9
:01084F0000A8
:0108500000A7
:0108510000A6
:0108520000A5
:0108530000A4
:0108540000A3
:0108550000A2
:0108560000A1
:0108570000A0
:01085800009F
:01085900009E
:01085A00009D
:01085B00009C
:01085C00009B
:01085D00009A
:01085E000099
:01085F000098
:010860000097
:010861000096
:010862000095
:010863000094
:010864000093
:010865000092
:010866000091
:010867000090
:01086800008F
:01086900008E
:01086A00008D
:01086B00008C
:01086C00008B
:01086D00008A
:01086E000089
:01086F000088
:010870000087
:010871000086
:010872000085
:010873000084
:010874000083
:010875000082
:010876000081
:010877000080
:01087800007F
:01087900007E
:01087A00007D
:01087B00007C
:01087C00007B
:01087D00007A
:01087E000079
:01087F000078
:010880000077
:010881000076
:010882000075
:010883000074
:010884000073
:010885000072
:010886000071
:010887000070
:01088800006F
:01088900006E
:01088A00006D
:01088B00006C
:01088C00006B
:01088D00006A
:01088E000069
:01088F000068
:010890000067
:010891000066
:010892000065
:010893000064
:010894000063
:010895000062
:010896000061
:010897000060
:01089800005F
:01089900005E
:01089A00005D
:01089B00005C
:01089C00005B
:01089D00005A
:01089E000059
:01089F000058
:0108A0000057
:0108A1000056
:0108A2000055
:0108A3000054
:0108A4000053
:0108A5000052
:0108A6000051
:0108A7000050
:0108A800004F
:0108A900004E
:0108AA00004D
:0108AB00004C
:0108AC00004B
:0108AD00004A
:0108AE000049
:0108AF000048
:0108B0000047
:0108B1000046
:0108B2000045
:0108B3000044
:0108B4000043
:0108B5000042
:0108B6000041
:0108B7000040
:0108B800003F
:0108B900003E
:0108BA00003D
:0108BB00003C
:0108BC00003B
:0108BD00003A
:0108BE000039
:0108BF000038
:0108C0000037
:0108C1000036
:0108C2000035
:0108C3000034
:0108C4000033
:0108C5000032
:0108C6000031
:0108C7000030
:0108C800002F
:0108C900002E
:0108CA00002D
:0108CB00002C
:0108CC00002B
:0108CD00002A
:0108CE000029
:0108CF000028
:0108D0000027
:0108D1000026
:0108D2000025
:0108D3000024
:0108D4000023
:0108D5000022
:0108D6000021
:0108D7000020
:0108D800001F
:0108D900001E
:0108DA00001D
:0108DB00001C
:0108DC00001B
:0108DD00001A
:0108DE000019
:0108DF000018
:0108E0000017
:0108E1000016
:0108E2000015
:0108E3000014
:0108E4000013
:0108E5000012
:0108E6000011
:0108E7000010
:0108E800000F
:0108E900000E
:0108EA00000D
:0108EB00000C
:0108EC00000B
:0108ED00000A
:0108EE000009
:0108EF000008
:0108F0000007
:0108F1000006
:0108F2000005
:0108F3000004
:0108F4000003
:0108F5000002
:0108F6000001
:0108F7000000
:0108F80000FF
:0108F90000FE
:0108FA0000FD
:0108FB0000FC
:0108FC0000FB
:0108FD0000FA
:0108FE0000F9
:0108FF0000F8
:0109000000F6
:0109010000F5
:0109020000F4
:0109030000F3
:0109040000F2
:0109050000F1
:0109060000F0
:0109070000EF
:0109080000EE
:0109090000ED
:01090A0000EC
:01090B0000EB
:01090C0000EA
:01090D0000E9
:01090E0000E8
:01090F0000E7
:0109100000E6
:0109110000E5
:0109120000E4
:0109130000E3
:0109140000E2
:0109150000E1
:0109160000E0
:0109170000DF
:0109180000DE
:0109190000DD
:01091A0000DC
:01091B0000DB
:01091C0000DA
:01091D0000D9
:01091E0000D8
:01091F0000D7
:0109200000D6
:0109210000D5
:0109220000D4
:0109230000D3
:0109240000D2
:0109250000D1
:0109260000D0
:0109270000CF
:0109280000CE
:0109290000CD
:01092A0000CC
:01092B0000CB
:01092C0000CA
:01092D0000C9
:01092E0000C8
:01092F0000C7
:0109300000C6
:0109310000C5
:0109320000C4
:0109330000C3
:0109340000C2
:0109350000C1
:0109360000C0
:0109370000BF
:0109380000BE
:0109390000BD
:01093A0000BC
:01093B0000BB
:01093C0000BA
:01093D0000B9
:01093E0000B8
:01093F0000B7
:0109400000B6
:0109410000B5
:0109420000B4
:0109430000B3
:0109440000B2
:0109450000B1
:0109460000B0
:0109470000AF
:0109480000AE
:0109490000AD
:01094A0000AC
:01094B0000AB
:01094C0000AA
:01094D0000A9
:01094E0000A8
:01094F0000A7
:0109500000A6
:0109510000A5
:0109520000A4
:0109530000A3
:0109540000A2
:0109550000A1
:0109560000A0
:01095700009F
:01095800009E
:01095900009D
:01095A00009C
:01095B00009B
:01095C00009A
:01095D000099
:01095E000098
:01095F000097
:010960000096
:010961000095
:010962000094
:010963000093
:010964000092
:010965000091
:010966000090
:01096700008F
:01096800008E
:01096900008D
:01096A00008C
:01096B00008B
:01096C00008A
:01096D000089
:01096E000088
:01096F000087
:010970000086
:010971000085
:010972000084
:010973000083
:010974000082
:010975000081
:010976000080
:01097700007F
:01097800007E
:01097900007D
:01097A00007C
:01097B00007B
:01097C00007A
:01097D000079
:01097E000078
:01097F000077
:010980000076
:010981000075
:010982000074
:010983000073
:010984000072
:010985000071
:010986000070
:01098700006F
:01098800006E
:01098900006D
:01098A00006C
:01098B00006B
:01098C00006A
:01098D000069
:01098E000068
:01098F000067
:010990000066
:010991000065
:010992000064
:010993000063
:010994000062
:010995000061
:010996000060
:01099700005F
:01099800005E
:01099900005D
:01099A00005C
:01099B00005B
:01099C00005A
:01099D000059
:01099E000058
:01099F000057
:0109A0000056
:0109A1000055
:0109A2000054
:0109A3000053
:0109A4000052
:0109A5000051
:0109A6000050
:0109A700004F
:0109A800004E
:0109A900004D
:0109AA00004C
:0109AB00004B
:0109AC00004A
:0109AD000049
:0109AE000048
:0109AF000047
:0109B0000046
:0109B1000045
:0109B2000044
:0109B3000043
:0109B4000042
:0109B5000041
:0109B6000040
:0109B700003F
:0109B800003E
:0109B900003D
:0109BA00003C
:0109BB00003B
:0109BC00003A
:0109BD000039
:0109BE000038
:0109BF000037
:0109C0000036
:0109C1000035
:0109C2000034
:0109C3000033
:0109C4000032
:0109C5000031
:0109C6000030
:0109C700002F
:0109C800002E
:0109C900002D
:0109CA00002C
:0109CB00002B
:0109CC00002A
:0109CD000029
:0109CE000028
:0109CF000027
:0109D0000026
:0109D1000025
:0109D2000024
:0109D3000023
:0109D4000022
:0109D5000021
:0109D6000020
:0109D700001F
:0109D800001E
:0109D900001D
:0109DA00001C
:0109DB00001B
:0109DC00001A
:0109DD000019
:0109DE000018
:0109DF000017
:0109E0000016
:0109E1000015
:0109E2000014
:0109E3000013
:0109E4000012
:0109E5000011
:0109E6000010
:0109E700000F
:0109E800000E
:0109E900000D
:0109EA00000C
:0109EB00000B
:0109EC00000A
:0109ED000009
:0109EE000008
:0109EF000007
:0109F0000006
:0109F1000005
:0109F2000004
:0109F3000003
:0109F4000002
:0109F5000001
:0109F6000000
:0109F70000FF
:0109F80000FE
:0109F90000FD
:0109FA0000FC
:0109FB0000FB
:0109FC0000FA
:0109FD0000F9
:0109FE0000F8
:0109FF0000F7
:010A000000F5
:010A010000F4
:010A020000F3
:010A030000F2
:010A040000F1
:010A050000F0
:010A060000EF
:010A070000EE
:010A080000ED
:010A090000EC
:010A0A0000EB
:010A0B0000EA
:010A0C0000E9
:010A0D0000E8
:010A0E0000E7
:010A0F0000E6
:010A100000E5
:010A110000E4
:010A120000E3
:010A130000E2
:010A140000E1
:010A150000E0
:010A160000DF
:010A170000DE
:010A180000DD
:010A190000DC
:010A1A0000DB
:010A1B0000DA
:010A1C0000D9
:010A1D0000D8
:010A1E0000D7
:010A1F0000D6
:010A200000D5
:010A210000D4
:010A220000D3
:010A230000D2
:010A240000D1
:010A250000D0
:010A260000CF
:010A270000CE
:010A280000CD
:010A290000CC
:010A2A0000CB
:010A2B0000CA
:010A2C0000C9
:010A2D0000C8
:010A2E0000C7
:010A2F0000C6
:010A300000C5
:010A310000C4
:010A320000C3
:010A330000C2
:010A340000C1
:010A350000C0
:010A360000BF
:010A370000BE
:010A380000BD
:010A390000BC
:010A3A0000BB
:010A3B0000BA
:010A3C0000B9
:010A3D0000B8
:010A3E0000B7
:010A3F0000B6
:010A400000B5
:010A410000B4
:010A420000B3
:010A430000B2
:010A440000B1
:010A450000B0
:010A460000AF
:010A470000AE
:010A480000AD
:010A490000AC
:010A4A0000AB
:010A4B0000AA
:010A4C0000A9
:010A4D0000A8
:010A4E0000A7
:010A4F0000A6
:010A500000A5
:010A510000A4
:010A520000A3
:010A530000A2
:010A540000A1
:010A550000A0
:010A5600009F
:010A5700009E
:010A5800009D
:010A5900009C
:010A5A00009B
:010A5B00009A
:010A5C000099
:010A5D000098
:010A5E000097
:010A5F000096
:010A60000095
:010A61000094
:010A62000093
:010A63000092
:010A64000091
:010A65000090
:010A6600008F
:010A6700008E
:010A6800008D
:010A6900008C
:010A6A00008B
:010A6B00008A
:010A6C000089
:010A6D000088
:010A6E000087
:010A6F000086
:010A70000085
:010A71000084
:010A72000083
:010A73000082
:010A74000081
:010A75000080
:010A7600007F
:010A7700007E
:010A7800007D
:010A7900007C
:010A7A00007B
:010A7B00007A
:010A7C000079
:010A7D000078
:010A7E000077
:010A7F000076
:010A80000075
:010A81000074
:010A82000073
:010A83000072
:010A84000071
:010A85000070
:010A8600006F
:010A8700006E
:010A8800006D
:010A8900006C
:010A8A00006B
:010A8B00006A
:010A8C000069
:010A8D000068
:010A8E000067
:010A8F000066
:010A90000065
:010A91000064
:010A92000063
:010A93000062
:010A94000061
:010A95000060
:010A9600005F
:010A9700005E
:010A9800005D
:010A9900005C
:010A9A00005B
:010A9B00005A
:010A9C000059
:010A9D000058
:010A9E000057
:010A9F000056
:010AA0000055
:010AA1000054
:010AA2000053
:010AA3000052
:010AA4000051
:010AA5000050
:010AA600004F
:010AA700004E
:010AA800004D
:010AA900004C
:010AAA00004B
:010AAB00004A
:010AAC000049
:010AAD000048
:010AAE000047
:010AAF000046
:010AB0000045
:010AB1000044
:010AB2000043
:010AB3000042
:010AB4000041
:010AB5000040
:010AB600003F
:010AB700003E
:010AB800003D
:010AB900003C
:010ABA00003B
:010ABB00003A
:010ABC000039
:010ABD000038
:010ABE000037
:010ABF000036
:010AC0000035
:010AC1000034
:010AC2000033
:010AC3000032
:010AC4000031
:010AC5000030
:010AC600002F
:010AC700002E
:010AC800002D
:010AC900002C
:010ACA00002B
:010ACB00002A
:010ACC000029
:010ACD000028
:010ACE000027
:010ACF000026
:010AD0000025
:010AD1000024
:010AD2000023
:010AD3000022
:010AD4000021
:010AD5000020
:010AD600001F
:010AD700001E
:010AD800001D
:010AD900001C
:010ADA00001B
:010ADB00001A
:010ADC000019
:010ADD000018
:010ADE000017
:010ADF000016
:010AE0000015
:010AE1000014
:010AE2000013
:010AE3000012
:010AE4000011
:010AE5000010
:010AE600000F
:010AE700000E
:010AE800000D
:010AE900000C
:010AEA00000B
:010AEB00000A
:010AEC000009
:010AED000008
:010AEE000007
:010AEF000006
:010AF0000005
:010AF1000004
:010AF2000003
:010AF3000002
:010AF4000001
:010AF5000000
:010AF60000FF
:010AF70000FE
:010AF80000FD
:010AF90000FC
:010AFA0000FB
:010AFB0000FA
:010AFC0000F9
:010AFD0000F8
:010AFE0000F7
:010AFF0000F6
:010B000000F4
:010B010000F3
:010B020000F2
:010B030000F1
:010B040000F0
:010B050000EF
:010B060000EE
:010B070000ED
:010B080000EC
:010B090000EB
:010B0A0000EA
:010B0B0000E9
:010B0C0000E8
:010B0D0000E7
:010B0E0000E6
:010B0F0000E5
:010B100000E4
:010B110000E3
:010B120000E2
:010B130000E1
:010B140000E0
:010B150000DF
:010B160000DE
:010B170000DD
:010B180000DC
:010B190000DB
:010B1A0000DA
:010B1B0000D9
:010B1C0000D8
:010B1D0000D7
:010B1E0000D6
:010B1F0000D5
:010B200000D4
:010B210000D3
:010B220000D2
:010B230000D1
:010B240000D0
:010B250000CF
:010B260000CE
:010B270000CD
:010B280000CC
:010B290000CB
:010B2A0000CA
:010B2B0000C9
:010B2C0000C8
:010B2D0000C7
:010B2E0000C6
:010B2F0000C5
:010B300000C4
:010B310000C3
:010B320000C2
:010B330000C1
:010B340000C0
:010B350000BF
:010B360000BE
:010B370000BD
:010B380000BC
:010B390000BB
:010B3A0000BA
:010B3B0000B9
:010B3C0000B8
:010B3D0000B7
:010B3E0000B6
:010B3F0000B5
:010B400000B4
:010B410000B3
:010B420000B2
:010B430000B1
:010B440000B0
:010B450000AF
:010B460000AE
:010B470000AD
:010B480000AC
:010B490000AB
:010B4A0000AA
:010B4B0000A9
:010B4C0000A8
:010B4D0000A7
:010B4E0000A6
:010B4F0000A5
:010B500000A4
:010B510000A3
:010B520000A2
:010B530000A1
:010B540000A0
:010B5500009F
:010B5600009E
:010B5700009D
:010B5800009C
:010B5900009B
:010B5A00009A
:010B5B000099
:010B5C000098
:010B5D000097
:010B5E000096
:010B5F000095
:010B60000094
:010B61000093
:010B62000092
:010B63000091
:010B64000090
:010B6500008F
:010B6600008E
:010B6700008D
:010B6800008C
:010B6900008B
:010B6A00008A
:010B6B000089
:010B6C000088
:010B6D000087
:010B6E000086
:010B6F000085
:010B70000084
:010B71000083
:010B72000082
:010B73000081
:010B74000080
:010B7500007F
:010B7600007E
:010B7700007D
:010B7800007C
:010B7900007B
:010B7A00007A
:010B7B000079
:010B7C000078
:010B7D000077
:010B7E000076
:010B7F000075
:010B80000074
:010B81000073
:010B82000072
:010B83000071
:010B84000070
:010B8500006F
:010B8600006E
:010B8700006D
:010B8800006C
:010B8900006B
:010B8A00006A
:010B8B000069
:010B8C000068
:010B8D000067
:010B8E000066
:010B8F000065
:010B90000064
:010B91000063
:010B92000062
:010B93000061
:010B94000060
:010B9500005F
:010B9600005E
:010B9700005D
:010B9800005C
:010B9900005B
:010B9A00005A
:010B9B000059
:010B9C000058
:010B9D000057
:010B9E000056
:010B9F000055
:010BA0000054
:010BA1000053
:010BA2000052
:010BA3000051
:010BA4000050
:010BA500004F
:010BA600004E
:010BA700004D
:010BA800004C
:010BA900004B
:010BAA00004A
:010BAB000049
:010BAC000048
:010BAD000047
:010BAE000046
:010BAF000045
:010BB0000044
:010BB1000043
:010BB2000042
:010BB3000041
:010BB4000040
:010BB500003F
:010BB600003E
:010BB700003D
:00000001FF
